:100000002BC60BC00AC009C008C007C01BC615C656
:1000100004C003C002C001C000C000001895959A3A
:10002000E3D69498E1D6959800000000089594983E
:10003000959800000000089594989598D5D6959AC3
:10004000D3D60000000008951F932F93949A10E8D0
:10005000212F2023203051F4959AC6D69498C4D6E7
:10006000949AC2D61695103099F707C09598BCD6C9
:100070009498BAD6949AB8D6F5CFB6D6949A95985D
:100080002F911F9130D008951F932F93949A18E0C9
:1000900000E0000000000000949800000000000054
:1000A00020B326FF02C0016001C00E7F949A1A950A
:1000B000103019F08894001FEFCF00002F911F918E
:1000C0000895959A91D694988FD6949A8DD69598AE
:1000D000000000000895959887D6949885D6949A44
:1000E0000000000008951F9300E094987DD610B39F
:1000F0001074103409F001E0949A000000001F9180
:1001000008952F93202F98DF9FDF00FF0FC0012F4E
:100110009BDF00FF0BC090DF022F016095DF00FF27
:1001200005C0B2DFD8DF7BDF80E001C08FEF2F9109
:10013000089582DF89DF00FF0AD0012F85DF00FFED
:1001400006D0022F81DF00FF02D069DF089501E0B1
:1001500010E09BD604EC10E020E07BD605ED10E02B
:1001600020E477D6909A00009098FCCF08952F93C2
:1001700020E01F931A95110F010F1F911A951F3F31
:1001800079F05ADF0F9360DF4ADF1F931A95103022
:1001900011F0000FFBCF202B1F910F910250EECFDB
:1001A000022F2F91089543E050E001E010E06DD65A
:1001B0000AE110E026E04DD6403041F403E210E0C1
:1001C00020E447D64F9350FDB1D14F91413041F4D7
:1001D00003E310E020E43DD64F9350FDC8D24F9189
:1001E000423041F405EE10E020E433D64F9350FD49
:1001F00036D44F91433041F409EF10E020E429D682
:100200004F9350FD96D44F9114D650FDCCCF552727
:100210005BD6083029F44395443009F44427C5CF10
:10022000043031F44A954F3F01F644E04A95BDCF82
:10023000023011F45FEFB9CF013031F74EC51F9393
:100240002F93102F00E01A301CF0005F1A50FBCFE4
:10025000010F2F911F9108951F932F930F93102F2C
:1002600012951F7020E00AE0103019F0200F1A9547
:10027000FBCF0F910F70020F2F911F9108950F93D5
:1002800006B30F70013069F1023059F1083019F0EE
:10029000043091F0F5CF4BD00F9103950F930F7071
:1002A0000A3011F00F9103C00F91005F007F021719
:1002B00009F4012F10E018C03AD00F91101741F443
:1002C000022F0A95202F2F702F3049F4065007C0B7
:1002D0000A950F930F700F300F9109F4065010E03C
:1002E00003C025D0102F0F9108950F9306B30F7000
:1002F0000130C9F00230B9F0083019F0043049F08B
:10030000F5CF15D00F910395021709F4012F10E0D6
:100310000DC00DD00F91101719F4022F0A9501C0CE
:100320000A9510E0E1CF03D0102F0F9108950F939D
:1003300009B7026009BF65D509B70D7F09BF0F91E5
:10034000AA9808950F931F932F93EF93FF9323E0A1
:1003500014E000EAD6DE0F93007F0295005D4DD0D9
:100360000F910F70005D49D02A95203021F00AE3EB
:1003700044D01A95EECF00E240D000EA16E0C1DE8C
:100380000F93007E0295202F02E418E02ED3E02F79
:10039000F12FC895002D31D03196C895002D2DD064
:1003A00000E22BD000EA15E0ACDE0F730F93007F64
:1003B0000295005D22D00F910F70005D1ED000E20B
:1003C0001CD00F910F7148DF0A95000F000F202FEE
:1003D00009E418E00AD3E02FF12F14E0C895002DAE
:1003E0000CD031961A951030C9F700E206D0FF9173
:1003F000EF912F911F910F9108955D9BFECF0CB946
:1004000008951F9303951F70105D0F9307D50F91EB
:100410000A951F9112951F70105D00D50895EF93F6
:10042000FF930F931F93202F0CE318E0DED2E02FF1
:10043000F12F1F910F91C895202D012F18E00395E2
:100440001A95103081F0269538F01F931FE50F9311
:10045000E5D40F911F91F3CF1F931AE20F93DED4CF
:100460000F911F91ECCFFF91EF9108952F930F9370
:10047000212F107F1295105DD1D40F910395122F6B
:100480001F70105DCBD42F9108952F930F93007F91
:100490000295005DB2DF0F910F70005DAEDF2F910E
:1004A00008952F931F93EF93FF930F9301E618E0A6
:1004B00020E09BD2E02FF12FC895002D003019F0DD
:1004C0009CDF3196F9CF0F910F93007F0295B7DE35
:1004D000102F007F0295005D90DF012F0F70005DEF
:1004E0008CDF00E28ADF0AE388DF00E286DF0F911B
:1004F000017000FD03C000E010E002C00FE110E059
:100500000EBB1FBBE09A0CB300FDFDCF0DB3003056
:1005100041F073DF0EB30395003091F71FB31395CD
:10052000EFCFFF91EF911F912F91089501E010E01F
:10053000ACD403E210E020E08CD40DE710E020E41E
:1005400088D406E41AE05AD200EA14E0DADD202F5B
:1005500070D408E4122FFDD0022F10E024E28FDEC9
:10056000202F1030A9F31F9300EA14E0E2DD1F9161
:10057000123009F0FBC000EA14E0DBDD5AD404E8D5
:1005800010E020E466D408E418E038D200EA13E072
:10059000B8DD202F4ED409E4122FDBD0022F10E05B
:1005A00020E66DDE202F1030A9F31F9300EA13E040
:1005B000C0DD1F91123009F0D9C000EA13E0B9DDA7
:1005C00038D40DE810E020E444D406E41AE016D252
:1005D00000EA16E096DD0F71202F2BD4122F07E4CE
:1005E000B8D0022F11E023E14ADE202F1030A9F30A
:1005F0001F9300EA16E085DD007E202B00EA16E05E
:1006000098DD1F91123009F0B1C000EA16E079DDE3
:10061000007E202B00EA16E08CDD0BD404E910E00C
:1006200020E417D400EA15E06CDD0F73202F01D40D
:10063000122F0EE48ED0022F11E022E320DE202FB5
:100640001030A9F31F9300EA15E05BDD007C2F93C7
:10065000202B00EA15E06DDD2F911F91123009F07B
:1006600085C000EA15E04DDD007C202B00EA15E096
:1006700060DDDFD301EA10E020E4EBD300EA16E00E
:1006800040DD007E02950695202FD3D32F93220FB5
:1006900002E418E0AAD1E02FF12FC8953196102D71
:1006A0000DE4BCD3C895102D0EE4B8D32F91022FC2
:1006B00010E027E0E4DD202F103039F31F9300EA2B
:1006C00016E01FDD0F712F932295220F202B00EAD9
:1006D00016E02FDD2F911F91123009F047C000EA7C
:1006E00016E00FDD0F712295220F202B00EA16E095
:1006F00020DD9FD303EB10E020E4ABD307E412E34B
:100700008DD3039510E38AD300EA1FEFFADC97DD5F
:10071000202F8FD309E4122F1CD0022F10E029E9DB
:10072000AEDD202F1030A9F3022F96DD202F2F935E
:1007300000EA1FEFFEDC00EA15E0E3DC0F732F9107
:1007400023702295220F220F202B00EA15E0F1DC06
:100750000DC01F93107F1295105D0F935FD30F9103
:100760001F911F70105D039559D30895089530E0CF
:100770000E2D0030A1F40F2D003089F401E010E0BF
:1007800084D302E410E020E064D302E510E020E42A
:1007900060D34FD399D30130E9F74BD3089500E0EC
:1007A0001FE02CD10EE510E020E053D342D33431CA
:1007B000F1F23F3F11F434E13A95032F40DD102F61
:1007C0000EE054DE2BE7032F2B5F0A950F3FE1F776
:1007D00020930001F0E0E0E6122F25E002EA20304D
:1007E00029F08FDC019313952A95F8CFF0E0E0E62D
:1007F00024E000E01191010F2A952030D9F70095EF
:100800000F5F1081011731F00BE2029300E00293B9
:1008100002930293E0E6119100E428DE1AE302E479
:10082000FDD203E4119122DE05E410E2F7D220812B
:100830002B5008F025EF255F21930F931F93022F74
:1008400015E4EDDD1F910F910DE413E0D7D03CD3FB
:10085000083011F43395AACF043011F43A95A6CF9D
:10086000013009F4A0C0023091F7E3D20CE003603C
:1008700010E00BD3E0E6F0E02081DBD2122F00E4A1
:10088000F5DD022F10E024E2FADC202F1030A9F36E
:1008900021932081CED2122F03E4E8DD022F10E055
:1008A00020E6EDDC202F1030A9F321932081C1D266
:1008B000022F15E4B4DD008110E02BE016DD00838B
:1008C000202F1030A1F301E010E0DFD20AE010E0A9
:1008D00020E0BFD201910081007F0295B0DC102F93
:1008E0000BE4C4DDA6D222E4008100FF04C00FE1C6
:1008F00010E0AFD203C000E010E0ABD2E5D2083088
:1009000021F4008101600083EDCF043021F40081E7
:100910000E7F0083E7CF023029F78BD20081007F62
:100920000295202F8CDC102F0BE4A0DD022F6DD15F
:10093000003021F40EE410E271D203C00EE41AE29A
:100940006DD2022F10E02FE02395CFDC1F9302958C
:1009500010811F70102B10831F911030F1F269D29B
:100960000CE010E092D20CE610E020E472D2ACD29F
:100970000830B1F4E0E6F0E01091000120E00191D0
:10098000200F2F93202F02EAD4DB3BD22F91139517
:10099000E436A9F720952F5F02EACBDB32D2FFCEF7
:1009A000043029F7FCCE0ED308950F931F932F9395
:1009B00010E000E4202F0F9313953EDB45DB00FF92
:1009C00004C000E041DB00FFC2DB29DB0F911830DF
:1009D00011F00E5FF0CF203721F000E710E0202F5C
:1009E000EACF2F911F910F910895110F8894001F46
:1009F00008F41395020F08F4139508952F93212FEF
:100A000010E20F930BD20F9103952A952030C1F776
:100A10002F9108950F931F932F9310E020E000E48F
:100A20000F931F9309DB10DB00FF04C00894279588
:100A3000F6DA02C0889427951F910F910E5F1395E7
:100A4000183009F0EDCF003829F000E710E0E22E71
:100A500020E0E6CFF22E2F911F910F91089501E033
:100A600010E013D204EF10E020E0F3D104EF10E027
:100A700020E4EFD104E411E4D1D108E028E01E2DF8
:100A8000889417951F9318F41AE2C8D102C01DE28A
:100A9000C5D11F9103952A95203091F7003521F09B
:100AA00008E428E01F2DECCF0FD20130E9F7C1D1C7
:100AB0000895FF93EF932F931F930F93E02FF12F40
:100AC0002191203081F12A952F930191DEDC0AE3F8
:100AD00094DC0191DADC00E290DC0191EF93FF936A
:100AE000202F0CE318E081DFE02FF12FC895002DB7
:100AF000FF91EF9118E01A95103059F006950F9379
:100B000020F00DE27ADC0F91F6CF0AE276DC0F914D
:100B1000F2CF00E272DC0191C4DC0AE06EDC0DE091
:100B20006CDC2F91CECF0F911F912F91EF91FF9100
:100B300008950F931F932F9301E010E0A6D10AE0D0
:100B400010E020E086D110E00BE490DC0CE00360C4
:100B500010E09BD100E00F9322E400FF04C00FE1FE
:100B600010E077D103C000E010E073D162D1ACD1C6
:100B7000083019F40F910F6FEECF043019F40F9174
:100B80000027E9CF023091F720E02F9352D12F9127
:100B9000122F0BE46BDC2F93022F5EDB36D0102F6D
:100BA0000EE4103019F410E239D102C01AE236D145
:100BB0002F91022F10E026E162DB202F2F931030BF
:100BC00029F30AE011E020E444D133D17DD108308B
:100BD00091F40F91202F22953FDB1F911170212B53
:100BE000B1DB0F93022F5DDC0DE007DC0AE005DCD2
:100BF0000F9126D202C00F910F910CE010E045D169
:100C000018D12F911F910F9108951F932F9303FDDA
:100C100007C01E2D21E0003059F00A95220FFBCFAE
:100C20001F2D077021E0003019F00A95220FFBCF2D
:100C30001223012F2F911F9108950F9300E802BFF7
:100C40000F9118957FEF0F931F9304E313ED0DBDE4
:100C50001CBD1F910F91189507E50DBF02E00EBF57
:100C600000EF07BB0FEB01BB0FEF0ABB04BB00E0BB
:100C70000BBB08BB05BB02BB07E109B908E00AB919
:100C800002E003BF00E802BF03E00EBD00E00FBDBD
:100C900004E313ED0DBD1CBD00E809BF789480E0AE
:100CA000BED9A2D0C4D9A0D00CE010E0EED008E3A9
:100CB000ECD0C2D900EAC8D900FF49DA00E0C4D9B3
:100CC00000FF45DA00E0C0D900FF41DAA8D97AD1A7
:100CD00000EB10E0EEDE9EDE68DE01E010E0D5D035
:100CE00006B3000000000F70023011F420DB5BCA75
:100CF0007030B1F300EA12E004DA003031F4F1D0E0
:100D000000EA12E0FED90030D9F304E010E020E060
:100D1000A0D022E01EE000EA1F93122FF2D91F910B
:100D200023952F93212F102F022F13DD2F91253084
:100D300031F002501AE372D0102F1250ECCF00EABB
:100D400016E0DFD9007E0295202F02E418E04DDE88
:100D5000E02FF12F00E4C895102D60D03196C89592
:100D6000102D03955BD000EA15E0CBD90F73102F3F
:100D700003E4EFDC00EA16E0C4D90F716DDA0A95DE
:100D8000000F000F202F09E418E02FDEE02FF12FD5
:100D900024E006E4C895102D41D0319603952A959C
:100DA0002030C1F70BE412E339D0039510E336D0BD
:100DB00000EA1FEFA6D90F9342DA102F0DE4C9DC29
:100DC00000EA15E09ED902950695069503702F91CD
:100DD000122F2370021739F0139516FD1127212FBA
:100DE00000EA1FEFA6D97CCF0F931F9311E004E018
:100DF0000A95F1F71A9511F004E0FACF1F910F91BF
:100E000008950F931F9310E800E00A95F1F71A95E3
:100E100011F000E0FACF1F910F9108950F931F93E7
:100E2000006810E032D01F91012F11E02ED00F91F9
:100E300008950F931F9304E00A95003039F0E1DF25
:100E400016B31F701030C1F304E0F6CF1F910F915D
:100E500008950EBB1FBB022F006810E016D020D0F3
:100E600011E0E09A0CB300FDFDCF0DB3003061F04E
:100E70000CD016D00EB303950EBB003019F40FB38F
:100E800003950FBB2395E7CF08950BBB129515BBB8
:100E9000106415BB1F7B15BB112715BB01D008952E
:100EA0000F931F9300E00ABB02E0029505BB0064AC
:100EB00005BB000019B30F7B05BB17FDF5CF0FEF86
:100EC0000ABB1F910F91089506B30F70013039F0DE
:100ED000023029F0083019F0043009F0F5CF27DA94
:100EE00008950F931F932F93EF93FF93222700EB07
:100EF00010E01ED0003009F415C01F930F9322DAC2
:100F00000F910F93CEDA0DE078DA0AE076DA0F91DE
:100F1000102F007F02951F7093D01F911030212F4A
:100F200009F0E5CFFF91EF912F911F910F91089557
:100F3000E02FF12F0F931F93122F2191211B110FDF
:100F4000110FE10F203009F436C000EA14E0D9D8BF
:100F50001191011719F0ED5F2A95F4CF00EA13E023
:100F6000D0D81191011719F0EE5F2A95EBCF00EA66
:100F700016E0C7D8007E0295069511E0003019F002
:100F8000110F0A95FBCF0191EF93FF932F931F93BE
:100F9000202F0CE318E029DDE02FF12F1F912F9176
:100FA000C895002DFF91EF91012311F0008104C03D
:100FB000EF5F2A95C7CF0027FF91EF9110812A9507
:100FC000121B08950F931F932F9300E810E020EB5E
:100FD00004D02F911F910F910895EF93FF932F93BA
:100FE000C22FD12F2196102F24E12F9324E02A9590
:100FF00002EA87D8099313952030C9F700271F9379
:1010000014E01A952A91020F1030D9F700950F5F5E
:101010001F91202F02EA75D81395201709F4CC5F91
:101020002F912A95203009F70C2F0A9510EB011B00
:10103000069506952F91C22F0883FF91EF91089591
:101040002F931F9303FF05C00770000F10E7010FD8
:1010500003C0000F10E4010F1F912FEF10FF222794
:10106000122FEAD7F1D700FF05C0012FEDD700FFFF
:101070006ED8D5D72F9108950001020408102040A2
:101080001F607F004D6F54755765546846725361F9
:1010900053754A616E20466562204D7263684170E7
:1010A00072204D6179204A756E654A756C7941757B
:1010B0006720536570204F6374204E6F762044651F
:0C10C00063204368616E6E656C200000C8
:00000001FF
